:020000040000FA
:020000000528D1
:08000800DC298B13831606307E
:100010009F001F3085008601870101308100831217
:100020008B1686018701A601A701A801A901AA01D3
:10003000AB01AC01AD01AE01AF01B001B101851260
:10004000A2297621051C2821851CF420051DA42049
:10005000851D1B21051E2D202128A617A6177621F8
:10006000051A4728261B442826174030B4000730BD
:10007000B500051D6620851D4D20D321B50B3928FF
:100080007920B40B37284B282613A6120710CA2153
:100090007621051E4728A6130800792085196328B4
:1000A000AF0A0A302F02031C5C28AF01B00A0630E9
:1000B0003002031C5C28B0010F30B6007920B60B6B
:1000C0005E28851D50284030B400080079200519AD
:1000D0007628B10A18303102031C6F28B1010F30A5
:1000E000B6007920B60B7128051D69284030B40090
:1000F00008008715261B8714A61986280C303102A4
:10010000031C842807158F2885168F288717310828
:1001100009248713071731088723071397288717A0
:1001200031086523871307173108E3220713871661
:1001300030084F22871207162F084F220712871107
:10014000851207118710080076210519CF28A614FB
:10015000AB282612A614AB01AC01AD01AE01CA2139
:10016000D820051DAB28851DAB280D30A4003530E7
:10017000A5002616D820051DCE28851DA928051EF8
:10018000C428261ECF28BA28CA217621A61ECB282D
:100190002613A6120710051EC428BA282612AB0182
:1001A000AC01AD01AE01CA217621051DD32808009E
:1001B000261B8714A61CDF288715851607158717A9
:1001C0002E089922871307172D084F220713871629
:1001D0002C084F22871207162B084F22071287116F
:1001E0008512071187100800762185181A29290819
:1001F000053C031904292908003C03190C29CA21CC
:100200007621851CFF281A298B132615AA0A183077
:100210002A02031C0E29AA018B132615A801A90185
:10022000CA217621851C1029A7010D30A200353086
:10023000A3008B170800762185192729A61D2229DE
:10024000A6112329A615CA217621851D2329080078
:100250007621051839294030B4000730B500051D56
:100260005B21851D3A21D321B50B2F297621B40BB3
:100270002D2908007621851952298B132615A80AE5
:100280000A302802031C4B29A801A90A06302902BA
:10029000031C4B29A9010F30B6007621B60B4D295E
:1002A000851D3F294030B400A7010D30A200353034
:1002B000A3008B170800762105196D298B132615CD
:1002C000AA0A18302A02031C6629AA010F30B600B8
:1002D0007621B60B6829051D60294030B400A701BE
:1002E0000D30A2003530A3008B17080026198715A2
:1002F000261B8714A61984290C302A02031C822984
:1003000007158D2985168D2987172A080924871333
:1003100007172A0887230713952987172A086523B3
:10032000871307172A08E3220713871629084F2285
:100330008712071628084F22071287118512071106
:1003400087100800FF30B400FF30B5000715851294
:10035000051CBB29B50BA629B40BA429FF30B4009A
:10036000FF30B50007118516051CBB29B50BB22956
:10037000B40BB029A229D3210518A229071185128F
:10038000CA217621051CC0290D30A2003530A300FA
:100390008B1721280530B200D330B300B30BCE2920
:1003A000B20BCC2908001930B200D330B300B30B24
:1003B000D729B20BD5290800A000030EA1000B110C
:1003C000A30B082AA20B082A26150D30A2003530EF
:1003D000A300A70A3C302702031C082AA701A61E77
:1003E000F629B70BF6292613A6120710A80A0A3019
:1003F0002802031C082AA801A90A06302902031CA6
:10040000082AA901AA0A18302A02031C082AAA01EC
:10041000221D0C2AA2182611A61B222A261F222AD8
:10042000A61A222A2A083102031D222A290830028C
:10043000031D222A28082F02031D222AA6160714AC
:100440000A30B700261E4A2AA50B462AA40B462AC4
:10045000A6140D30A4003530A500AB0A0A302B02DB
:10046000031C462AAB01AC0A06302C02031C462AA8
:10047000AC01AD0A0A302D02031C462AAD01AE0ABA
:1004800006302E02031C462AAE012612241D4A2ADB
:10049000A418A610210E8300A00E200E0900B8009B
:1004A000003C0319782A3808013C03197B2A3808D4
:1004B000023C03197E2A3808033C0319812A3808B4
:1004C000043C0319842A3808053C0319872A380894
:1004D000063C03198A2A3808073C03198D2A380874
:1004E000083C0319902A3808093C0319932A962AD4
:1004F000FC308600962A60308600962ADA30860024
:10050000962AF2308600962A66308600962AB63001
:100510008600962ABE308600962AE4308600962A07
:10052000FE308600962AF6308600962AD321860170
:100530000800B800003C0319C22A3808013C03191E
:10054000C52A3808023C0319C82A3808033C031995
:10055000CB2A3808043C0319CE2A3808053C031975
:10056000D12A3808063C0319D42A3808073C031955
:10057000D72A3808083C0319DA2A3808093C031935
:10058000DD2AE02A00308600E02A60308600E02A7A
:10059000DA308600E02AF2308600E02A66308600F3
:1005A000E02AB6308600E02ABE308600E02AE43039
:1005B0008600E02AFE308600E02AF6308600E02A37
:1005C000D32186010800B800003C03194A2B3808E3
:1005D000013C0319472B3808023C03194A2B380801
:1005E000033C03194D2B3808043C0319502B3808E1
:1005F000053C0319532B3808063C0319562B3808C1
:10060000073C0319592B3808083C03195C2B3808A0
:10061000093C03195F2B38080A3C0319442B38089E
:100620000B3C0319472B38080C3C03194A2B38089C
:100630000D3C0319472B38080E3C03194A2B380888
:100640000F3C03194D2B3808103C0319502B380868
:10065000113C0319532B3808123C0319562B380848
:10066000133C0319592B3808143C03195C2B380828
:10067000153C03195F2B3808163C0319442B380826
:10068000173C0319472B622BFC308600622B60302D
:100690008600622BDA308600622BF2308600622BF5
:1006A00066308600622BB6308600622BBE30860034
:1006B000622BE4308600622BFE308600622BF6301F
:1006C0008600622BD32186010800B800003C031984
:1006D0007E2B38080A3C03197E2B38080B3C031983
:1006E0007E2B38080C3C03197E2B3808163C031966
:1006F0007E2B3808173C03197E2B812B6030860037
:10070000842B00308600842BD32186010800B8009A
:10071000003C0319E82B3808013C0319EB2B38087F
:10072000023C0319EE2B3808033C0319F12B38085F
:10073000043C0319F42B3808053C0319F72B38083F
:10074000063C0319FA2B3808073C0319FD2B38081F
:10075000083C0319002C3808093C0319032C3808FD
:100760000A3C0319E82B38080B3C0319EB2B38081B
:100770000C3C0319EE2B38080D3C0319F12B3808FB
:100780000E3C0319F42B38080F3C0319F72B3808DB
:10079000103C0319FA2B3808113C0319FD2B3808BB
:1007A000123C0319002C3808133C0319032C380899
:1007B000143C0319E82B3808153C0319EB2B3808B7
:1007C000163C0319EE2B3808173C0319F12B062CA5
:1007D000FC308600062C60308600062CDA3086005D
:1007E000062CF2308600062C66308600062CB630C9
:1007F0008600062CBE308600062CE4308600062CCF
:10080000FE308600062CF6308600062CD3218601A9
:100810000800B8000A3C0319422C38080B3C0319A5
:10082000422C38080C3C0319422C38080D3C0319A3
:10083000422C38080E3C0319422C38080F3C03198F
:10084000422C3808103C0319422C3808113C03197B
:10085000422C3808123C0319422C3808133C031967
:10086000422C3808143C0319452C3808153C031950
:10087000452C3808163C0319452C3808173C031939
:10088000452C482C603086004B2CDA3086004B2CEF
:0C089000003086004B2CD32186010800AC
:02400E00723FFF
:00000001FF
